:10000000F228A501A400B5172730A3001030142052
:100010000330A300E8301420A30164301420A301AE
:100020000A30142024081F28A2002508A100240853
:10003000A000BB202008031DB513B51B0800303EEF
:10004000A600380884000930A70003102C20A60C55
:10005000A70B262803142C288413B51D3B28000861
:100060003604351D36068000841700083604031C4C
:1000700036068000462800083604031C360635196B
:10008000360680008417360980054628350D063966
:10009000A0004F20A100A00A4F2000008E280030B1
:1000A0008A00200882070134753403341534003483
:1000B0003C340C34D9340F39A00083161F088F3913
:1000C00030389F0083120310A00DA00D1F08C13906
:1000D000200401389F000030A10032308E209F1490
:1000E0009F1870281E08A10083161E08ED2883168D
:1000F000F83881050F39810463000F308104ED2841
:10010000A301A200FF30A207031CA307031CED28D4
:100110000330A100DF308E208228A101E83EA0003C
:10012000A109FC30031C9728A00703189428A007F6
:100130006400A10F942820189D28A01CA12800006D
:10014000A1280800A2000330AB28A2000130AB2890
:10015000A2000630AB28A80023082102031DB22804
:100160002208200204300318013003190230280548
:10017000031DFF30ED28A501A4011030A600210DBC
:10018000A40DA50D2208A4022308031C230FA50219
:100190000318D1282208A40723080318230FA50752
:1001A0000310A00DA10DA60BBF282008ED281030CC
:1001B000A800A101A001A70CA60C031CE528220899
:1001C000A00723080318230FA107A10CA00CA50C5E
:1001D000A40CA80BDB282408ED2883130313831237
:1001E00064000800FF238316900083129F17831674
:1001F00038309F00831207309900A22103305B2022
:10020000C2002108C30006211D21FE284208A600C5
:100210004308A7003130A200A301D720B20025086F
:10022000B3003208A0003308A1006430A200A3018B
:10023000BB20BA002108BB0008003A08A0003B0818
:10024000A100A3012330A520031D3429C001C10151
:1002500005118316051183128512831685128312E8
:1002600044100430772094296400441843298516EB
:100270008316851283120515831605118312033028
:10028000A300E830812023303A02C0000030031C74
:10029000013E3B02C1004008A0004108A100A301AB
:1002A0000330A220031D57290330C000C1010130D3
:1002B000BE00BF013E08A0003F08A100A3013230EC
:1002C000A520031D93298516831685128312051513
:1002D0008316051183120130BC00BD013C08A0004B
:1002E0003D08A100A3010A30A520031D8F293C0869
:1002F000A0003D08A1004108A3004008A820031D5C
:10030000892905118316051183128512831685121A
:10031000831201308020BC0A0319BD0F6E29BE0A6A
:100320000319BF0F5A29441408000530B8000130E2
:10033000B6000630B5000A3020200D30202008001D
:100340006300A02905158316051183120730A30049
:10035000D030812005118316051183129521952136
:100360000530B8000130B6000630B500413020201D
:100370006C302020613020206E302020273020205B
:100380007330202020302020453020206C30202069
:1003900065302020633020207430202072302020EF
:1003A0006F3020206E3020206930202063302020E4
:1003B0002030202050302020723020206F3020202C
:1003C0006A302020653020206330202074302020C7
:1003D0007330202020302020493020206E30202013
:1003E000633020202E30202095210530B8000130C8
:1003F000B6000630B50050302020573020204D3058
:1004000020202030202054302020653020206D30E6
:100410002020703020206530202072302020613074
:10042000202074302020753020207230202065304C
:10043000202020302020433020206F3020206E30BC
:10044000202074302020723020206F3020206C302B
:1004500020206C3020206530202064302020203087
:10046000202046302020613020206E302020952131
:100470000530B8000130B6000630B5002D30202020
:100480002D3020202D3020202D3020202D302020F8
:100490002D3020202D3020202D3020202D302020E8
:1004A0002D3020202D3020202D3020202D302020D8
:1004B0002D3020202D3020202D3020202D302020C8
:1004C0002D3020202D3020202D3020202D302020B8
:1004D0002D3020202D3020202D3020202D302020A8
:1004E0002D302020952103305B20C2002108C3005D
:1004F000062195210530B8000130B6000630B50060
:10050000723020206130202077302020543020208D
:10051000653020206D302020703020204430202095
:100520006130202074302020613020203A3020209B
:10053000203020204308A50042080220203020203F
:10054000203020202030202020302020203020206B
:100550002030202063302020613020206C3020208B
:1005600063302020753020206C3020206130202026
:10057000743020206530202064302020543020202A
:10058000653020206D302020703020203A3020202F
:10059000203020203B08A5003A0802209521952113
:0205A000080051
:02400E00DC3F95
:00000001FF
